:020000040800F2
:1000000018460020790200089B3400089734000845
:1000100099340008191D0008D939000800000000B3
:100020000000000000000000000000007335000820
:10003000771D0008000000009D3400087535000899
:10004000930200089302000893020008930200083C
:10005000930200089302000893020008930200082C
:10006000930200089302000893020008930200081C
:100070001D1D0008291D00089302000893020008B6
:10008000351D0008411D0008930200089302000876
:1000900093020008930200089302000893020008EC
:1000A00093020008930200089302000893020008DC
:1000B00093020008930200089302000893020008CC
:1000C00093020008930200089302000893020008BC
:1000D000930200089302000851390008953900087E
:1000E000930200089302000893020008930200089C
:1000F000930200089302000893020008930200088C
:10010000930200089302000893020008930200087B
:10011000930200089302000893020008930200086B
:10012000930200089302000893020008930200085B
:1001300000F002F800F090F80AA090E8000C824469
:100140008344AAF10107DA4501D100F085F8AFF246
:10015000090EBAE80F0013F0010F18BFFB1A43F0A5
:1001600001031847F452000014530000103A24BF52
:1001700078C878C1FAD8520724BF30C830C144BF0C
:1001800004680C607047000000230024002500264E
:10019000103A28BF78C1FBD8520728BF30C148BFEA
:1001A0000B6070476E2900F02D83702900F0858464
:1001B000662905F00580652905F00280672904F0AD
:1001C000FF87612904F0FE8703681B0A28BF41F0FE
:1001D0008001692900F0C280642900F0BF80752980
:1001E00000F0BC806F2900F01384782900F051845E
:1001F000E92900F0AD83E42900F0AA83F52900F095
:10020000A783EF2900F01084F82900F050840368D8
:10021000DB0928BF41F08001632900F02E83732998
:1002200000F03383E32901F05F80F32901F064805B
:10023000002070471FB501F0B1F804000020002134
:1002400004F0A8FF401C60600020002104F08CFF37
:10025000E0601FBD10B510BD01F072F81146FFF748
:10026000E9FF04F0FBF901F04BF903B4FFF7F2FFEB
:1002700003BC01F08FF90000094880470948004796
:10028000FEE7FEE7FEE7FEE7FEE7FEE7FEE7FEE746
:10029000FEE7FEE704480549054A064B70470000A3
:1002A0007935000831010008184000201846002068
:1002B00018420020184200201CB50C46064B7B4417
:1002C00069460090204600F0B6FA044600206946D0
:1002D00000F0C4FA20461CBD9B0500000FB41CB5FD
:1002E000084B06AA7B4469460090059800F0A3FAE3
:1002F00004460020694600F0B1FA20461CBC5DF8B7
:1003000014FB00007505000070B50C460546012A77
:1003100005D02878800600D5EA69002302E0012391
:1003200005E05B1C934202D2E05C0028F9D1A86989
:10033000E618C01AA861286A18442862284600F006
:10034000CFF904E0D5E9012114F8010B9047B4423C
:10035000F8D3284600F0DAF970BD00002DE9F0412D
:100360000646002410687529314616A510D000F005
:10037000DEF9002802DA404213A507E031688A0757
:1003800001D512A502E0490704D511A5012401E019
:1003900000F0D6F900210A2206F1240709E0B0FB9B
:1003A000F2FCB0FBF2F302FB1C003030785418462C
:1003B000491C0028F3D123462A463046BDE8F041C7
:1003C00000F0C7B9000000002D0000002B00000065
:1003D000200000002DE9F05F894604464FF0000A36
:1003E000DFF874B1FB44C0F820A02046E1688847DC
:1003F000002874D0252806D0D4E901219047206A2E
:10040000401C2062F1E700265F462046E1688847ED
:100410002028054607DB312D05D2781910F8200C6D
:1004200008B10643F1E7B00701D526F00406C4F889
:100430001CA00027C4F818A02A2D09D0284603F0D4
:1004400003FB38B304EB8708303DC8F8185019E0B7
:1004500059F8041B204604EB87029161E168884744
:10046000012F054618D1E069002820DA26F0200681
:100470001DE0D8F8180000EB800005EB4000303894
:10048000C8F818002046E1688847054603F0DCFA02
:100490000028EED1012F0AD02E2D08D12046E16888
:1004A00088477F1C0546022F46F02006C4DBA06962
:1004B000002803DA404246F00106A061F00701D0AF
:1004C00026F010066C2D0BD0682D09D04C2D39D09C
:1004D0006A2D35D0742D35D07A2D33D016E038E022
:1004E000E1682F4620468847B842054609D16C2F5F
:1004F00026D04FF48060E1680643204688470546D1
:1005000004E06C2F1AD04FF4807006430DB3A5F1B0
:100510004100192802D8203546F400664A4629468B
:10052000204626604E46FFF73DFE80B101280BD0E5
:10053000F61D26F0070000F1080956E74020E4E721
:100540008020D8E70020D6E706F104094DE72846C9
:1005500052E7206ABDE8F09F0A4E000030B505461C
:100560000B462A4613F8014B12F8010B08B1A042C2
:10057000F8D01CB1002802D06D1CF1E7284630BD30
:1005800010B5431C02E010F8011B71B18107FAD1CC
:100590004FF0013202C88C1A8C4314EAC211F9D010
:1005A000C01A0A0603D0C01E10BDC01A10BD0A042E
:1005B00001D0801E10BD0902FCD0401E10BD032AD0
:1005C00040F2308010F0030C00F0158011F8013B70
:1005D000BCF1020F624498BF11F801CB00F8013B57
:1005E00038BF11F8013BA2F1040298BF00F801CB1B
:1005F00038BF00F8013B11F0030300F06982083AAC
:10060000C0F0088051F8043B083A51F804CBA0E848
:100610000810F5E7121D5CBF51F8043B40F8043B9D
:10062000AFF30080D20724BF11F8013B11F801CBD2
:1006300048BF11F8012B24BF00F8013B00F801CBA3
:1006400048BF00F8012B70474FF000020429C0F0AA
:10065000128010F0030C00F01B80CCF1040CBCF1F4
:10066000020F18BF00F8012BA8BF20F8022BA1EB46
:100670000C0100F00DB85FEAC17C24BF00F8012B2B
:1006800000F8012B48BF00F8012B70474FF0000223
:1006900000B5134694469646203922BFA0E80C5078
:1006A000A0E80C50B1F12001BFF4F7AF090728BF53
:1006B000A0E80C5048BF0CC05DF804EB890028BFCF
:1006C00040F8042B08BF704748BF20F8022B11F0F8
:1006D000804F18BF00F8012B704770477047704774
:1006E00070B5044685690068C10601D5302600E072
:1006F0002026C00707D070BDD4E9012130469047BD
:10070000206A401C20626D1EF6D570BD70B504468F
:1007100085690078C00707D170BDD4E90121202088
:100720009047206A401C20626D1EF6D570BD096896
:100730004A0501D540B27047C905FCD500B27047E3
:1007400009684A0501D5C0B27047C905FCD580B219
:1007500070472DE9F0470D4699469246044600F150
:1007600024080168880604D5E06921F010012160A1
:1007700000E00120A84201DD471B00E00027A1693D
:100780007A1902EB0900081AA0612078C00602D489
:100790002046FFF7A5FF002608E0D4E901211AF85A
:1007A00006009047206A401C761C20624E45F4DB10
:1007B0002078C0060AD52046FFF792FF06E0D4E96C
:1007C000012130209047206A401C2062381EA7F18A
:1007D0000107F4DC07E0D4E9012118F8050090478F
:1007E000206A401C2062281EA5F10105F3DC20468A
:1007F000FFF78CFF2078000602D50220BDE8F087C5
:100800000120FBE711680268006A530501D50870F2
:100810000AE0D30501D5088006E0130603D5C21708
:10082000C1E9000200E008600120704701694A1C2C
:1008300002610878704700B58FB0CDE90131002121
:10084000059105497944CDE9031011466846FFF743
:10085000C1FD0FB000BD0000E5FFFFFF0A6802F810
:10086000010B0A60704710B5436913B1AFF3008004
:1008700001E0FFF749FD012010BD127800F12401CD
:100880000A7000224A700122EDE711684FF0FF3232
:10089000E9E700002DE9FF5F15468A460446DFF8C8
:1008A000AC80F8440027D8E900103E46CDE900109E
:1008B00010E03AF816106A4602A800F021FD411C2B
:1008C00007D02178890603D5E269391891420DD8FD
:1008D0000744761C2078800602D5E069B84205DD21
:1008E000AE42E6DB3AF816000028E2D1A069C01B50
:1008F000A0612046FFF7F4FED8E90010CDE9001012
:10090000002017E03AF818106A4602A800F0F8FC38
:10091000B0F1FF3F81460BD000250DF1080B05E03B
:10092000D4E901211BF8050090476D1C4D45F7D314
:1009300008F10100B0428046E4DB206A38442062BE
:100940002046FFF7E3FEBDE8FF9F00005E49000080
:100950002DE9F0418046D21D22F007020025D2E9A0
:100960000002F52915A614D0011E72F1000106DA65
:100970000023D0EB030063EB020211A608E0D8F8D5
:1009800000108B0701D50FA602E0490701D50EA67E
:1009900001251146002408F1240704E000F0CAF8FC
:1009A00030323A55641C50EA0102F7D12B463246E8
:1009B00021464046BDE8F041FFF7CBBE00000000F5
:1009C0002D0000002B0000002000000030B40021AA
:1009D00000F1240408E002F00705D208303542EAAD
:1009E0004372DB086554491C52EA0305F3D10468DD
:1009F000002310A2250708D504F020040C4304D0DE
:100A0000C46901230CA2641EC46130BCFFF7A1BEFF
:100A100010B5044621461068FFF792FE02462046B4
:100A2000BDE810400023D1E7D21D22F00701D1E933
:100A30000023CBE70000000030000000F0B40D46BA
:100A40000188090502D5214C7C4402E01F4C7C44FE
:100A50000E34002100F1240608E002F00F0712090D
:100A6000E75D42EA03721B097754491C52EA030707
:100A7000F3D102780023120704D5702D06D009B1F6
:100A8000022311342246F0BCFFF763BE0123103469
:100A9000F8E770B504460D4621461068FFF750FE92
:100AA000024629462046BDE870400023C6E7D21D15
:100AB00022F00703D3E90023C0E70368126843F07C
:100AC000200303600823C3610023B7E7C047000089
:100AD00010B5203AC0F00B80B1E81850203AA0E8D9
:100AE0001850B1E81850A0E81850BFF4F5AF5FEA0D
:100AF000027C24BFB1E81850A0E8185044BF18C9C0
:100B000018C0BDE810405FEA827C24BF51F8043B66
:100B100040F8043B08BF7047D20728BF31F8023BBA
:100B200048BF11F8012B28BF20F8023B48BF00F84E
:100B3000012B704730B5B0F10A024FEA900E71F107
:100B400000034EEA817EB0EB0E0061EB91014FEAAB
:100B5000101E4EEA017E10EB0E0041EB11114FEA20
:100B6000102E4EEA016E10EB0E0041EB11214FEA00
:100B7000104E4EEA014E10EB0E0041EB11414018B1
:100B800041F100014FEAD00040EA41704FEAD10143
:100B900010EB80054FEA810444EA907444EB0104B1
:100BA0006D1944EB0404521BA3414FF0000348BFEE
:100BB0000A3200D530BD401C41F1000130BD704704
:100BC0002DE9FF4F0C461E464FF0FF378BB0D2E9A0
:100BD0000001DDF860800A908A46C1F30A5505B924
:100BE0003D46002108464FF00000BAF1000F00F426
:100BF000400005DA00EB80004FF4400101EA5000AC
:100C00004FEA9059B9F1010F00DDB9460A9850EA50
:100C10004A000ED044F61050A5F2FF3545432F147C
:100C2000B8F1000F1ED07542291E1EDDC9F1000269
:100C30001CE0B8F1010F4FF0000001D0302103E0BB
:100C4000F24305E02154401CB042FBDB3046002259
:100C5000002121540B99C1F80880C1E900200FB090
:100C6000BDE8F08FBD1B6D1CDEE74A4600DA694225
:100C700006A800F0D7FB06AB93E8070003AB83E8B8
:100C8000070050460A9900F08CFC8DE80700A0F59B
:100C900000501F3800900398002D09DD42F21F011B
:100CA0004A46084403A90390684600F0EBFE08E0BA
:100CB000A0F500504A461F3803A90390684600F08B
:100CC000F5FE8DE807000004000C03D04FF0FF3064
:100CD000410800E01046B8F1000F03D00022009256
:100CE00015461EE0751E05D4FFF724FF303262550D
:100CF0006D1EF9D5B3460122084302D000227F1CA5
:100D000004E02078302801D100227F1E002A0997B4
:100D100086D01DE0112D07DAFFF70CFF3032625547
:100D20006D1C50EA0102F5D1084302D00098C8B109
:100D30000EE00021681E05E0235C625C63542254CF
:100D4000401E491C8142F7DBAB46A81B401E0990A0
:100D5000002004F80B000B98099AC0F80880C0E93D
:100D6000002B7CE711264FF0000859E72DE9F04FE2
:100D700088460446D21D22F0070191B0D1E9000156
:100D8000CDE90A0102F029FE02460B98C00F01D0FE
:100D90002D2007E02068810701D52B2002E02021CB
:100DA00001EAC000032A099001D0072A05DB0346A7
:100DB0004146204600F0F6FA0BE12078800601D586
:100DC000E06900E00620B8F1650F814606D0B8F171
:100DD000660F18D0B8F1670F70D131E00020B9F17B
:100DE000110F009001DB112301E009F101030AAAB0
:100DF00001A90CA8FFF7E4FEDDE90C70002609F15B
:100E00000105834647E001204B4600904FF0004724
:100E10000AAA01A90CA8FFF7D3FEDDE90DB00C99D1
:100E20005D46002610B909F101000D18B9EB050067
:100E300003D4C0F1FF3609F10105A5EB09002BE051
:100E4000B9F1010F01DA4FF001090020B9F1110FDA
:100E50000090484601DD112300E003460AAA01A9DB
:100E60000CA8FFF7ADFEDDE90C704D460026834669
:100E7000207800070AD4AB4500DA5D4601A8012DB1
:100E800004DD411911F8011C302907D04F4502DA61
:100E900017F1040F04DA012082460FE06D1EEEE721
:100EA000002F02DCED1B3E4403E0781CA84200DD6D
:100EB0007D1CB81B00F1010A4FF0004720780007A5
:100EC00003D4AA4501DB4FF0FF3A0021B7F1004FF0
:100ED0000DF143088DF8431024D002202B23002F5E
:100EE00001DA7F422D230A21021EA0F1010000DC5D
:100EF0005FB197FBF1FC97FBF1F201FB1C7C1746FD
:100F00000CF1300C08F801CDEEE7A8F101000370F8
:100F10002188090501D5452100E06521A0F10108DE
:100F200000F8011C09980FA9A1EB0807FF1D00B1EB
:100F30000120411901EBEA70A1693844081A401EEA
:100F4000A0612078C00602D42046FFF7C9FB0998AB
:100F500028B1D4E901219047206A401C2062207802
:100F6000C00622D52046FFF7BBFB1EE0002E04DBA7
:100F7000B34502DD01A8805D00E03020D4E9012105
:100F80009047206A401C2062761CAAF101005FEAAB
:100F9000000A0AD100F002FAC0680168405CD4E996
:100FA00001219047206A401C2062281EA5F10105FE
:100FB000DCDC07E0D4E9012118F8010B9047206A36
:100FC000401C2062381EA7F10107F3DC2046FFF722
:100FD0009DFB032011B043E62DE9F04F04460D467A
:100FE000D21D22F0070089B0D0E90092484617468A
:100FF000394602F0F2FC0246F80F01D02D2307E03B
:101000002068810701D52B2302E0202101EAC003DB
:101010008DF820300BB1012000E00020032A824629
:1010200001D0072A04DB2946204600F0BBF93DE148
:101030002078800601D40D2500E0E569C7F30A5643
:101040000D2D49DA00214FEA175B08464FF00000EA
:10105000002F00F4400007DA00EB80004FF440015D
:1010600000EBD07001EA60008115012901DD4FF02D
:10107000FF3100224FEA850CBCF1180F06D313464E
:10108000ACF118004FF08052C24003E04FF48013DF
:1010900023FA0CF30CF10C0CBCF1200F04D3ACF1CF
:1010A000200C09FA0CF001E007FA0CF000294FF0CF
:1010B000004801DD18B90FE00ED140450CD319EB03
:1010C00002095F4121B9404502D19F4329EA020943
:1010D000BBEB175F00D0761C2088000502D57B484B
:1010E000784402E079487844193808AA302302F895
:1010F0000A30037C0AF10101002E0AF1020A53545E
:101100006A4602DC4FF0300101E04FF031014FF050
:1011100001088DF8001002D0A6F2FF3603E059EA6C
:10112000470100D06A4E002D02DC2178090704D562
:101130004FF002082E218DF80110C44600210BE06B
:10114000C7F303433F01C35C491C6D1E02F808301E
:10115000052908F1010801DA002DF1DC00210CE07D
:1011600000EB1973491C1B786D1E082902F8083022
:101170004FEA091908F1010801DA002DF0DC2178A5
:10118000890602D514E0A8F10108E04505DD02EB6F
:10119000080111F8011C3029F5D0B8F1000F07DD66
:1011A00002EB080111F8011C2E2901D1A8F1010858
:1011B000002D05DD3E2102F808106D1E08F1010822
:1011C000407C002E02F8080008F1010804DA2D2006
:1011D000764202F8080002E02B2002F808000A21FB
:1011E0004FF47A70864208F101080BDB96FBF0F3AE
:1011F000303302F8083096FBF0F308F1010800FBE9
:10120000136601E0642E0CDB642096FBF0F33033B0
:1012100002F8083096FBF0F308F1010800FB1366B2
:1012200001E00A2E06DB96FBF1F0303002F80800F0
:1012300008F1010896FBF1F001FB1060303002F874
:101240000800A16908F1010808EB050202EB0A0099
:10125000081AA0612078C00602D42046FFF740FAA1
:10126000216A08AE01EB0A00206204E0D4E9012102
:1012700016F8010B9047BAF1010AF7D22078C006A0
:1012800002D52046FFF72CFA6E4609E016F8010B4E
:101290003E280FD0D4E901219047206A401C2062EB
:1012A000B8F10108F2D22046FFF730FA09B0032066
:1012B000BDE8F08F206A2844206203E0D4E90121D0
:1012C000302090476D1EEBD3F8E70000634100002B
:1012D00002FCFFFF10B5436913B1AFF3008001E0DA
:1012E000FFF7D8FA012010BD128800F12401828492
:1012F0000022C2840122EDE711684FF0FF32E9E7D6
:1013000070B516460C46054600F040F8036893F8A1
:101310000101012806D0FF2C0FD8185D68B101200B
:101320002C7070BDD3F807013246214603F2071333
:1013300003442846BDE8704018474FF0FF3070BDA9
:10134000754600F0E3F8AE4605006946534620F0C6
:101350000700854618B020B5FEF79CFFBDE8204089
:101360004FF000064FF000074FF000084FF0000B61
:1013700021F00701AC46ACE8C009ACE8C009ACE814
:10138000C009ACE8C0098D467047000010B500F0F8
:1013900005F8001D10BD00BFFD3D0000004870476E
:1013A000D43F00202DE9F0411F4604460326016882
:1013B000072A01F4006004DB08B116A505E016A5B4
:1013C00003E008B115A500E015A521F0100020608C
:1013D000A069C01EA0610FB1401EA0612046FFF7AA
:1013E0007FF94FB1D4E9012138469047206A401C6B
:1013F0002062C01C206206E0206AFAE7D4E90121DD
:1014000015F8010B9047761EF8D22046FFF77EF9BB
:10141000BDE8F0814E414E006E616E00494E4600BF
:10142000696E66002DE9F047814616468AB033485A
:1014300078440DC88DE80D0030487844801C03AC1A
:101440000DC884E80D0041F69B300844372190FB1D
:10145000F1F290FBF1F5A5F1800501FB12041B3CB4
:1014600002D56442012000E00020DFF890A0804611
:101470000027FA44AAF1BE0A0DE0E00709D032467F
:10148000684607EB47010AEB810100F00FFB8DE88E
:10149000070064107F1C002CEFD1184F7F44AC3F35
:1014A00018E0E80714D007EB04100DF1180A90E8D3
:1014B0000E008AE80E00C068F04201D19819089029
:1014C000324606A903A800F0F1FA03AB83E807004F
:1014D0006D10641C002DE4D132466946B8F1000F4E
:1014E00003A802D000F0CEFA01E000F0DFFAC9E96B
:1014F0000001C9F808200AB0BDE8F087A43E00004A
:101500000446AFF300802046FEF7AFFE0048704768
:10151000B43F00204FF0013C50F8042B51F8043B3D
:101520009A4221D1A2EB0C03934313EACC1317D1B7
:1015300050F8042B51F8043B9A4215D1A2EB0C034E
:10154000934313EACC130BD150F8042B51F8043B0E
:101550009A4209D1A2EB0C03934313EACC13DBD0DC
:101560004FF00000704700BFD01A01BAB1FA81F104
:1015700001F0180122FA01F0CB40C1F12001DBB2E9
:10158000C0B2C01A2CFA01F3D11A914311EAC31167
:10159000E6D1704701491820ABBEFEE726000200E5
:1015A00070475FEA400C08BF91F0000F4FEA8C23B0
:1015B0004FEAC12243EA51514FEA1C5018BF00F5CF
:1015C000F0404FEA300018BF41F000415FEA6C5C28
:1015D00000F02980BCF1FF3F08BF40F08040704719
:1015E000130C06BF12044FF0100C4FF0000C130E3A
:1015F00004BF12020CF1080C130F04BF12010CF10E
:10160000040C930F04BF92000CF1020CD30F04BF23
:1016100052000CF1010C11464FF00002A0F11F0026
:10162000A0EB0C00704711F0004F08BF704731F07D
:1016300000413FF4D5AF0B0C06BF09044FF0100C6E
:101640004FF0000C0B0E04BF09020CF1080C0B0F3D
:1016500004BF09010CF1040C8B0F04BF89000CF1CD
:10166000020CCB0F04BF49000CF1010CCCF120039C
:10167000A0EB0C0022FA03F302FA0CF241EA030198
:1016800000F10100704720F07F4C80EA030023F056
:101690007F47ACEB070303F57C5300F0004003F1F8
:1016A000FF032DE980494FEA154B09B44FEA144373
:1016B00025EA0B4E24EA03480FF2042606EB132713
:1016C00049083E785FEA320203FB0667C7F5000768
:1016D00007FB06F64FEA54374FEAD64606F10206F4
:1016E00007FB066CCCF1005C4FEA1C472CEA074C68
:1016F00007FB06F40CFB06F504EB15464FEA9616BD
:1017000034BF00204FF000404FEAD13706FB07FC02
:101710004FEA1C4C0CFB0BF7D21B03FB0CF761EBE5
:1017200007010CFB0EF7B0EB074072EB17420CFB06
:1017300008F734BFA2EB0742B2EB074261EB174157
:101740004FEA0C444FEA910706FB07FC4FEA1C4C9A
:101750000CFB0BF7B0EBC74072EB573203FB0CF7F7
:1017600034BFA2EBC742B2EBC74261EB57310CFB6F
:101770000EF7B0EBC70072EB57720CFB08F734BFE3
:10178000A2EBC702B2EBC70261EB5771039F4FEAAE
:10179000816141EA921104EBCC044FEAD1374FEA60
:1017A000826206FB07FC42EA90124FEA80604FEA31
:1017B0001C4C0CFB0BF7D21B03FB0CF761EB070176
:1017C0000CFB0EF7B0EB074072EB17420CFB08F76F
:1017D00034BFA2EB0742B2EB074261EB17414FEA7D
:1017E0008C554FEA910704EB9C2406FB07FC4FEA5B
:1017F0001C4C0CFB0BF7B0EBC74072EB573203FBF2
:101800000CF734BFA2EBC742B2EBC74261EB5731D2
:101810000CFB0EF7B0EBC70072EB57720CFB08F72E
:1018200034BFA2EBC702B2EBC70261EB577115EBF5
:101830004C254FEA816141EA92114FEA82624FEAF8
:10184000D13742EA901206FB07FC44F100044FEA4C
:1018500080604FEA1C4C0CFB0BF7D21B03FB0CF710
:1018600061EB07010CFB0EF7B0EB074072EB174280
:101870000CFB08F734BFA2EB0742B2EB074261EB67
:10188000174115EB1C154FEA813141EA92414FEAAD
:10189000823242EA90424FEA80304FEA0C7644F1BD
:1018A000000448EA03434EEA0B484FF0000EB2EB47
:1018B000080C71EB030724BF624639464EEB0E0E4F
:1018C0004FF0000B0018524149414BEB0B0BB2EBB0
:1018D000080C71EB03077BF1000B24BF624639460D
:1018E0004EEB0E0E4FF0000B0018524149414BEBEE
:1018F0000B0BB2EB080C71EB03077BF1000B24BF61
:10190000624639464EEB0E0E51EA020718BF46F00A
:10191000010616EB0E7655F1000254F1000103D5D5
:10192000BDE88901BDE80088BDE88901BDE800483F
:10193000B619524141EB0101A3F1010370478080C8
:101940007F7E7D7C7B7A7978777676757473727119
:1019500071706F6E6E6D6C6C6B6A6A6968686766D1
:1019600066656464636362616160605F5F5E5E5D63
:101970005D5C5C5B5B5A5A595958585757565655D7
:1019800055555454535352525251515050504F4F39
:101990004F4E4E4D4D4D4C4C4C4B4B4B4A4A4A4989
:1019A00049494848484747474746464645454544CC
:1019B0004444444343434342424242414141002B59
:1019C00026D4770021D01CB54FEA370703B44FF077
:1019D00010004FF010014FF000000FBCBDE81040A8
:1019E0000BF1010BBBF1010F08BF5FEA170722BF24
:1019F00012F1010211F101014FF0004143F1000326
:101A000000F0004043EA00007047F9D35708DAE7D6
:101A100046EA064613F1400F4FEA16461FDD13F162
:101A2000200FDFBF16430A46002120335B42C8D097
:101A3000C3F1200746EA064602FA07F74FEA1646C0
:101A400046EA0706C3F1200722FA03F201FA07F774
:101A500021FA03F14FF0000342EA0702B1E746EA38
:101A6000020646EA06464FEA164646EA0106BCBFAB
:101A700046EA0646360C4FF000034FF000024FF0E6
:101A800000019EE72DE9C048934630B491E8380044
:101A900007C831EA400C48BF34EA430C03D5FFF7CE
:101AA000F2FDFFF78CFFF0BCBDE800882DE9C048CF
:101AB000934630B491E8380007C810F0804F08BF53
:101AC00013F0804F03D100F005F8FFF778FFF0BC6A
:101AD000BDE8008820F07F4780EA030023F07F4CB8
:101AE00007EB0C03A3F57C5300F00040A3F1FE03C9
:101AF00092F0000F00F0B38095F0000F00F07780B7
:101B00002DE901494FEA11404FEA144621EA004805
:101B100000FB06FC24EA064708FB06F607FB08F86C
:101B200000FB07F718EB06484CEB164C4FEA124B3C
:101B300018EB07484FEA15464CEB174022EA0B4ECC
:101B40000BFB06FC25EA06470EFB06F607FB0EFE1E
:101B50000BFB07F71EEB064E4CEB164C4FF0000646
:101B60001EEB074E4CEB174B18EB0B0840F1000037
:101B700018EB0E0B58EB000840F100008F1A4FF0E5
:101B800000013CBFC943661B14BFB5EB040C002128
:101B90003CBFC943F61B4FEA17444EEA8E0E27EAB4
:101BA00004454FEA1C4704FB07622CEA074C05FB7F
:101BB00007F70CFB05F604FB0CFC16EB074642EBA3
:101BC000174216EB0C4642EB1C421BEB060658EB89
:101BD0000202414146EA9E0601D5BDE80189B619D7
:101BE000524141EB0101A3F10103BDE801894FEA34
:101BF00014454FEA114724EA054621EA074C05FB44
:101C000007F406FB07F70CFB06F105FB0CFC11EBD8
:101C1000074144EB17444FEA124711EB0C4144EBE8
:101C20001C4422EA074C05FB07F206FB07F70CFBF6
:101C300006F605FB0CFC16EB074642EB174216EBCB
:101C40000C4642EB1C456A1854F1000148BF70472E
:101C5000B619524141EB0101A3F10103704795F020
:101C6000000F37D04FEA11424FEA144721EA0246EB
:101C700024EA074C02FB07F106FB07F70CFB06F40E
:101C800002FB0CFC14EB074441EB17414FEA1547EC
:101C900014EB0C4441EB1C4125EA074C02FB07F511
:101CA00006FB07F70CFB06F602FB0CFC16EB0746DF
:101CB00045EB174516EB0C4645EB1C42121951F14A
:101CC000000148BF7047B619524141EB0101A3F131
:101CD000010370474FEA14454FEA114724EA0546CD
:101CE00021EA074C05FB07F106FB07F70CFB06F2A0
:101CF0004FF0000605FB0CFC12EB074241EB1741CD
:101D000012EB0C4251EB1C4148BF7047921841EB5B
:101D10000101A3F101037047FEE70000014800F054
:101D2000E9B80000941A0020014800F0E3B8000070
:101D3000501A0020014800F0DDB8000064070020C0
:101D4000014800F0D7B80000A807002030B590F88F
:101D500040500124AC40C56B6C600468636043680C
:101D6000102B036803D099600068C26030BD9A6090
:101D70000068C16030BD704772B6FEE710B590F8DC
:101D800021100022022905D00421816380F820203F
:101D9000012010BD01680B6823F00E030B60016881
:101DA0000B6823F001030B6090F84030C46B0121F5
:101DB00001FA03F3636080F8211080F820201046B8
:101DC00010BD00002DE9F05F90F8211000240229D9
:101DD00003D004218163012485E001680A6822F0B0
:101DE0000E020A6001680A6822F001020A603F4E92
:101DF0003E4FB215DFF8F4C0DFF8F090DFF8ECA04A
:101E0000DFF8E8B0DFF8E4E00168783F130115027D
:101E1000ACF1640CA9F15009AAF13C0AABF1280B12
:101E2000AEF1140E4FF48018B14227D9B9420ED04A
:101E3000614512D049451DD0514518D0594518D09B
:101E4000714501D1424615E0294EB14201D101222E
:101E500010E0274E1436B14201D110220AE0244E80
:101E60002836B14206D0224A3C32914201D11A466C
:101E700000E02A461E49091F0A602BE0B94213D030
:101E8000614517D0494522D051451DD059451DD037
:101E9000714501D142461AE0B14202D14FF0807241
:101EA00015E0134EB14201D1012210E0104E14365C
:101EB000B14201D110220AE00D4E2836B14206D0BF
:101EC0000B4A3C32914201D11A4600E02A460749AA
:101ED00080394A60012180F82110002180F820100B
:101EE000416B01B188472046BDE8F09F8000024069
:101EF000080402402DE9F05FC16B0A6801680B68B5
:101F0000046C4FF0040808FA04F8844D844E854FA1
:101F1000DFF814C2DFF81492DFF814A2DFF814B26D
:101F2000DFF814E218EA020F65D05FEA437862D561
:101F30000A68920603D40A6822F004020A60DFF8F5
:101F4000F0814FF48062016808F114081301140253
:101F5000414524D9A9420DD0B1420FD0B9421AD07F
:101F6000614515D0494515D0514501D1120312E004
:101F7000594501D104220EE0714501D140220AE009
:101F80006D4D1435A94206D06B4A2832914201D1D9
:101F90001A4600E022466749091F0A6029E0A94263
:101FA00013D0B14215D0B94220D061451BD049456C
:101FB0001BD0514502D14FF4800217E0414502D1B8
:101FC0004FF0806212E0594501D104220EE07145C4
:101FD00001D140220AE0584D1435A94206D0564A94
:101FE0002832914201D11A4600E022464B49083975
:101FF0004A60C16A71E04FF0020808FA04F818EA72
:10200000020F70D05FEA83786DD50A68920606D415
:102010000A6822F00A020A60012180F82110DFF824
:1020200010814FF40072016808F1140813011402C2
:10203000414524D9A9420DD0B1420FD0B9421AD09E
:10204000614515D0494515D0514501D1120312E023
:10205000594501D102220EE0714501D120220AE04A
:10206000354D1435A94206D0334A2832914201D168
:102070001A4600E022462F49091F0A6029E0A942BA
:1020800013D0B14215D0B94220D061451BD049458B
:102090001BD0514502D14FF4001217E0414502D147
:1020A0004FF0007212E0594501D102220EE0714555
:1020B00001D120220AE0204D1435A94206D01E4A43
:1020C0002832914201D11A4600E0224613490839CC
:1020D0004A60002180F82010816A00291CD0BDE8E8
:1020E000F05F0847FFE70825A540154214D01A07FE
:1020F00012D50A6822F00E020A6090F84020C36BE5
:10210000012101FA02F25A60816380F82110002156
:1021100080F82010016BE0E7BDE8F09F0800024066
:102120001C000240300002404400024058000240BF
:102130006C000240080402401C04024030B560B14B
:102140001A4B026814219A4209D2194B1344B3FB6B
:10215000F1F18900016417490AE0012030BD134BF9
:102160005B421344B3FBF1F1890001640F49083964
:10217000C163022180F82110136843F6F0718B438C
:10218000F0E901142143D0E902452C4321430469BD
:10219000214344692143846921431943116000218B
:1021A0004163012242770177084630BD08040240AE
:1021B000F8FFFDBF0000024070B5044690F8200013
:1021C000002501280CD0012084F8200094F821601B
:1021D0000020012E06D084F820000225284670BD7C
:1021E000022070BD022684F82160A0632068066882
:1021F00026F0010606602046FFF7A8FDE06A0028E9
:102200002068016802D041F00E0106E021F00401CF
:1022100001602068016841F00A01016020680168DE
:1022200041F001010160D9E770B5044600F01CF9E6
:102230000546601C02D004480078044400F014F9FC
:10224000401BA042FAD370BD0C0000202DE9F84FCE
:10225000DFF8C8910024A9F1040B23460F2709F1E8
:10226000040AABF1040ED1E00125A54006EA0502FF
:10227000AA4276D1DFF8A8C14E68A6EB0C086645E5
:102280002BD00DDC032E34D005DC36B3012E19D053
:10229000022E2FD11BE0112E16D0122E2AD119E0BA
:1022A000B8F5881F19D006DCB8F5803F15D0B8F511
:1022B000801F1FD111E0B8F5001F0ED0B8F5041F24
:1022C00018D10AE0CB6815E0CB681B1D12E0CB6883
:1022D00008330FE0CB680C330CE08B682BB1012B7B
:1022E0004FF0080303D0456104E0042302E00561D8
:1022F00000E00023FF2A01D8064601E000F10406B1
:102300004FEA840501D9A5F12005D6F8008007FA27
:1023100005FC28EA0C0803FA05F548EA0508C6F8A2
:1023200000804D68ED0070D53E4DAE6946F0010667
:10233000AE61AD6924F0030605F0010500953A4D44
:1023400006EB050CDCF80850A607360F07FA06F86E
:1023500025EA0805DFF8D480404503D14FF0000896
:1023600025E052E0DFF8C880404502D14FF0010877
:102370001DE0DFF8C080404502D14FF0020816E0B2
:10238000DFF8B480404502D14FF003080FE0DFF8DA
:10239000AC80404502D14FF0040808E0DFF8A0808F
:1023A000404502D14FF0050801E04FF0060808FA59
:1023B00006F848EA0508CCF808804D68D9F80060AE
:1023C000ED024D4601D5164300E096432E604D6860
:1023D000DAF80060AD02554601D5164300E0964399
:1023E0002E604D68DBF80060AD035D4601D51643F5
:1023F00000E096432E604D68DEF80060ED03754600
:1024000001D5164300E096432E60641C0A68164608
:10241000E2407FF429AFBDE8F88F000008040140D6
:1024200000001110001002400000014000080140AF
:10243000000C014000100140001401400018014050
:10244000001C01408068084000D001207047C2682D
:1024500021EA02030A4043EA0241016170470AB1DE
:10246000016170470904FBE701488068704700007C
:102470000C00002002488168027811448160704796
:102480000C000020074810B5016841F01001016000
:10249000032000F075F80F2000F006F800F024F893
:1024A000002010BD0020024070B50D4D04464FF4D1
:1024B0007A712878B1FBF0F00A490968B1FBF0F0B5
:1024C00000F082FB48B9102C07D200222146501E92
:1024D00000F036F800206C6070BD012070BD000077
:1024E0000C000020180000200C4808B5816941F05C
:1024F00001018161816901F001010091C16941F02F
:102500008051C161C06900F080500090044841686A
:1025100021F0E06141F00071416008BD001002400F
:1025200000000140002809DB00F01F02012191405A
:102530004009800000F1E020C0F800117047000061
:10254000F0B40E4B1B680C46C3F30223C3F107051E
:10255000042D00D90425191D072901D2002300E00C
:10256000DB1E012606FA05F1491E214099409E40D6
:10257000761E16403143F0BC01F043BA0CED00E08A
:10258000064900F0070208684FF6FF03184040EACA
:102590000220034A10430860704700000CED00E081
:1025A0000000FA052DE9F0470F46050061D0434EC3
:1025B000306800F00700B84209D2306820F0070008
:1025C00038433060306800F00700B84251D12868C5
:1025D0003B4C810712D5400703D5606840F4E060AA
:1025E00060602878000703D5606840F46050606040
:1025F0006068A96820F0F000084360602878C00790
:1026000028D06868012810D02168022810D08907D6
:1026100000292EDA616821F0030101436160FFF7B0
:1026200023FF804641F288390DE021688903EFE7F6
:102630008901EDE7FFF718FFA0EB0801494502D932
:102640000320BDE8F0876068696800F00C00B0EB1B
:10265000810FEFD1306800F00700B8420BD9306825
:1026600020F0070038433060306800F00700B842BF
:1026700001D00120E5E72878400705D56068E968C2
:1026800020F4E060084360602878000706D56068A1
:10269000296920F4605040EAC100606000F038F819
:1026A0006168084AC1F30311515CC84006490860DB
:1026B00006480068FFF7F8FE0020C2E7002002404D
:1026C00000100240DA51000818000020100000201D
:1026D0000448054900684968044AC1F30221515C75
:1026E000C84070471800002000100240EA5100085E
:1026F0000448054900684968044AC1F3C221515C95
:10270000C84070471800002000100240EA5100083D
:102710000E4A51680E4801F00C03042B11D0082B0F
:102720000FD10C48C1F38343C903C05C0AD551687B
:10273000084AC1F34041921E515C054A5043B0FB28
:10274000F1F0704704494843704700000010024010
:1027500000127A00CA51000800093D002DE9F84F27
:10276000040070D02078C04DC00749D06868C0F31D
:102770008100012807D06868C0F38100022809D1D0
:102780006868C00306D52868800339D560680028CA
:10279000E7D035E06068B0F5803F0BD010B1B0F500
:1027A000A02F11D0286820F480302860286820F4F9
:1027B000802002E0286840F480302860606890B192
:1027C000FFF752FE06460AE0286840F480202860A1
:1027D000F0E700BFFFF748FE801B642873D8286825
:1027E0008003F7D50CE0FFF73FFE064605E000BF8B
:1027F000FFF73AFE801B6428F0D828688003F7D4DE
:1028000020789A4E80074FF001094FF0000839D523
:10281000686810F00C0F07D06868C0F381000228C8
:1028200009D16868C00306D42868800714D52069D8
:10283000012808D110E02069B0B1C6F80090FFF778
:1028400013FE074605E00AE1FFF70EFEC01B022853
:10285000C4D828688007F7D52868616920F0F80097
:1028600040EAC10028600DE0C6F80080FFF7FCFDDB
:10287000074604E0FFF7F8FDC01B022823D82868AC
:102880008007F7D4207800072CD57948A169D9B101
:10289000C0F80090FFF7E8FD074604E0FFF7E4FD0D
:1028A000C01B02280FD8686A8007F7D571484FF41B
:1028B000FA510068B0FBF1F0009000BF0098411E93
:1028C0000091FAD20EE080E0C0F80080FFF7CCFD66
:1028D000074604E0FFF7C8FDC01B022875D8686AE8
:1028E0008007F7D42078400760D5E8690027C0004A
:1028F00008D4E86940F08050E861E869012700F0F9
:10290000805000905C480168C90513D40168834673
:1029100041F480710160FFF7A7FD824606E000BF29
:10292000FFF7A2FDA0EB0A0064284ED8DBF80000F8
:10293000C005F5D5E06801280AD008B1052813D0F4
:10294000286A20F001002862286A20F0040002E0D2
:10295000286A40F001002862E06841F2883B98B1A3
:10296000FFF782FD82460BE0286A40F004002862EF
:10297000EEE700BFFFF778FDA0EB0A0159455AD8F2
:10298000286A8007F6D50CE0FFF76EFD824605E069
:10299000FFF76AFDA0EB0A0159454CD8286A800769
:1029A000F6D41FB1E86920F08050E861E06988B38F
:1029B0006968C1F38101022944D00228C6F8608009
:1029C00004D0FFF751FD044638E034E0FFF74CFD3A
:1029D000074604E0FFF748FDC01B02282BD82868F3
:1029E0008001F7D4206AB0F5803F05D16868A168FE
:1029F00020F4003008436860D4E90801084369689E
:102A000021F4741108436860C6F86090FFF72CFD4C
:102A1000044606E025E000BFFFF726FD001B022864
:102A200009D828688001F7D51BE000BFFFF71CFD1F
:102A3000001B022802D90320BDE8F88F2868800116
:102A4000F4D40EE00128F7D06868226A00F48031DF
:102A5000914204D1616A00F47010884201D00120D3
:102A6000EAE70020E8E700000010024000004242D0
:102A700080044242180000200070004070B504003D
:102A800009D0606A002540B125616561A56294F8AE
:102A9000510040B10CE0012070BD6068B0F5827F4C
:102AA000F4D0E561F2E784F85050204600F040F899
:102AB000022084F851002068016821F04001016083
:102AC000A088218900F4827001F404410843A1899F
:102AD00001F400610843217C01F002010843217DDB
:102AE00001F001010843218B01F400710843217FAB
:102AF00001F03801084394F8201001F080010843E8
:102B0000218D01F40051084321680860A069042167
:102B100001EA1040216848602068C16921F4006121
:102B2000C1616565012084F85100002070BD00007E
:102B30002DE9F041054600681E491F4C0226012779
:102B400086B04FF00308884216D1A06940F0040017
:102B5000A061A06900F004000490A06940F48050D6
:102B6000A061A069694600F480500490E0208DE8DF
:102B7000C1011248FFF76AFB11492868884216D143
:102B8000A06940F00800A061A06900F0080004906E
:102B9000E06940F48040E061E06900F48040049026
:102BA00088008DE8C10169460648FFF74FFB06B073
:102BB000BDE8F081003001400010024000080140F3
:102BC00000380040000C014010B5401EB0F1807F7D
:102BD00001D3012010BD4FF0E02460610F21601788
:102BE00000F00FFF0020A06107202061002010BD31
:102BF000704700002DE9F041074600683049002584
:102C000088422DD12F4C304E54F8140B616F304454
:102C10004860FFF729FC54F8741F886020680C3066
:102C200044F8080B54F89019884203D12548103015
:102C3000C4F8880020684FF40072C0F5005191423A
:102C400004D3D4F888103044086003E02560D4F839
:102C500088000660D4F8880001681C4800F034FB46
:102C60001B493868884228D11A481B490268D0F8A5
:102C700088300A445A60D0F888200C32C0F8882086
:102C8000D0F890309A4203D100F11002C0F88820A9
:102C90000268C2F50063FF2B01D9114400E0056012
:102CA000D0F888201160D0F888004FF48072016855
:102CB000BDE8F041094800F007BBBDE8F081000025
:102CC00000480040F0180020D81E0020081A0020FC
:102CD0000044004004060020EC0F00201C070020E8
:102CE00070B5044620680C3050E8001F21F4907144
:102CF00040E80012002AF5D12068143050E8001F87
:102D000021F0010140E80012002AF5D1206B0128D2
:102D100009D120680C3050E8001F21F0100140E874
:102D20000012002AF5D1206840694FF020024106C8
:102D30004FF0000015D52168143151E8003F23F011
:102D4000400341E80035002DF5D1E16B49B1094858
:102D50004863E06BFFF736F850B1E06B416B884792
:102D600006E0E08584F8422020632046FFF742FF1A
:102D7000002070BD7936000870470000F8B5016882
:102D800004460868CA684B6910F00F0F4FF0000541
:102D90005AD003F0010602F49077374365D0C1079B
:102DA00005D0D10503D5616C41F001016164410793
:102DB00005D5D90703D0616C41F002016164810738
:102DC00005D5D90703D0616C41F0040161640107A6
:102DD00007D502F02001314303D0616C41F00801B6
:102DE0006164616C00293BD0800604D5900602D551
:102DF000204600F0A7FC20684069616CC0F3801099
:102E000001F00801014320462BD000F066FC206849
:102E10004069400621D52068143050E8001F21F099
:102E2000400140E80012002AF5D1E06BA8B16D49DD
:102E30004163E06BFEF7C6FF002811D0E06B416BE9
:102E400001B0BDE8F040084783060ED593060CD5C7
:102E50002046BDE8F84000F075BC2046FFF78CFF27
:102E6000F8BDFFF789FF6564F8BD266B2023012EAE
:102E70007CD1C6067AD5D60678D508684868009011
:102E800048694FF00206400640D5E16B086840688B
:102E90000004000CE8D0A28D8242E5D9E085886963
:102EA00020282DD020680C3050E8001F21F48071BC
:102EB00040E80012002AF5D12168143151E8000FD2
:102EC00020F0010041E80002002AF5D1206814300A
:102ED00050E8001F21F0400140E80012002AF5D11F
:102EE00084F84230256320680C3050E8001F21F040
:102EF000100140E80012002AF5D1E06BFEF73EFF1A
:102F00006663A08DE18D401A81B22AE0A08DE18D2B
:102F1000401A81B2E08D0028A6D00029A4D02268F2
:102F20000C3252E8000F20F4907042E80007002FA6
:102F3000F5D12068143050E8002F22F0010240E85B
:102F40000027002FF5D184F84230256320680C302B
:102F500050E8002F22F0100240E80023002BF5D1AA
:102F600066632046FFF744FEF8BDFFE705062BD554
:102F7000150629D594F841002128F5D1A068B0F5AF
:102F8000805F01D12069B0B1206A411C21622168B3
:102F900000784860E08C401E0004000CE084E3D11F
:102FA0002068C16821F08001C1602068C16841F0DB
:102FB0004001C160D8E7206A0088C0F3080048607B
:102FC000206A801C2062E5E74006CDD55006CBD5AF
:102FD000CA68204622F04002CA6084F8413000F0FE
:102FE0003BFAC1E77B35000870B5040004D094F8C3
:102FF0004100002510B106E0012070BD84F840506A
:10300000204600F023F8242084F841002068C1689D
:1030100021F40051C160204600F0F6FB20680169F0
:1030200021F4904101612068416921F02A01416148
:103030002068C16841F40051C1606564202084F8B3
:10304000410084F842006563002070BD2DE9F04F17
:10305000044601689148DFF84892924E0227002505
:1030600085B04FF00308814220D1B06940F00400E0
:10307000B061B06900F004000490B06940F4804091
:10308000B061B069CDF80C8000F480400490481520
:10309000CDE9000769464846FFF7D8F83015CDE975
:1030A0000005694648460295FFF7D0F87E4920683A
:1030B0004FF0800A884275D1B06940F00400B061D9
:1030C000B06900F004000490F06940F40030F06151
:1030D000F06900F400300490706940F00100706104
:1030E0007069694600F0010004900420CDE90007F2
:1030F000CDF80C804846FFF7A9F80820CDE9000577
:10310000694648460295FFF7A1F8022200212620D1
:10311000FFF716FA2620FFF705FADFF894B16349A6
:103120000BF5D470CBF8A4111021A0E822044FF4C1
:10313000005940F81059456185610BF5D270CBF804
:10314000C0910490FEF7FAFF08B1FEF715FE04984F
:10315000A063564958461439CBF8C841E0E95815E0
:10316000C0E9025A0561456185615248CBF87C91FE
:103170008146FEF7E3FF08B1FEF7FEFDC4F83C9080
:10318000002211461020CBF88441FFF7D9F9102016
:10319000FFF7C8F9002211461120FFF7D1F91120DD
:1031A000FFF7C0F944492068884273D1B06940F004
:1031B0000800B061B06900F008000490F06940F4C4
:1031C0008020F061F06900F480200490706940F084
:1031D000010070617069394E00F00100049008151B
:1031E000CDE900076946CDF80C803046FFF72EF890
:1031F000F014CDE90005694630460295FFF726F840
:10320000022200212720FFF79BF92720FFF78AF9E8
:1032100026482B4E64385746C6F8A40106F5D476E6
:103220001020A1C64FF4005820C6264820C681466B
:1032300066E86F58FEF782FF08B1FEF79DFD1B4858
:10324000C4F838905038C6F8C841C6E95805C6E9F0
:103250005A57C6F87051C6F87451C6E95E581948F5
:1032600044380546FEF76AFF08B1FEF785FDE563C1
:10327000002211460C20C6F88441FFF761F90C20AA
:10328000FFF750F9002211460D20FFF759F90D20E4
:10329000FFF748F905B0BDE8F08F000000380140A5
:1032A000000801400010024000440040800002403D
:1032B000040600206407002000480040000C014084
:1032C000F0180020941A002090F84230202B01D0F2
:1032D0000220704721B11AB10023036300F0F0BA55
:1032E000012070472DE9F041074600683349002569
:1032F000884231D1324C334E54F8140B00F5007033
:1033000044F8140C616F30444860FFF7ADF854F88E
:10331000741F886020680C3044F8080B54F890192A
:10332000884203D126481030C4F8880020684FF442
:103330000072C0F50051914204D3D4F88810304493
:10334000086003E02560D4F888000660D4F888009F
:1033500001681D48FFF7B8FF1C49386888422BD127
:103360001B481C49026802F580720260D0F8883060
:103370000A445A60D0F888200C32C0F88820D0F86F
:1033800090309A4203D100F11002C0F88820026800
:10339000C2F50063FF2B01D9114400E00560D0F8AD
:1033A00088201160D0F888004FF480720168BDE871
:1033B000F0410948FFF788BFBDE8F08100480040B0
:1033C000F0180020D81E0020081A002000440040F9
:1033D00004060020EC0F00201C07002070470000AE
:1033E00070B5044690F84100202801D0022070BD3D
:1033F00049B342B32162A284E284002060642123A5
:1034000084F84130A56B114BAB62A56B104BEB629E
:10341000A56B104B2B63A36B5863256813462A1DBD
:10342000A06BFEF7C9FE21686FF0400008602068BD
:10343000143050E8001F41F0800140E80012002ADB
:10344000F5D1002070BD012070BD00008F3600084E
:10345000D13600088B35000870B50446006809496C
:103460000025884204D1084E3573FEF7FDFFB06099
:1034700006492068884204D1054C2573FEF7F4FF05
:10348000A06070BD00480040F018002000440040DB
:10349000040600207047FEE7FEE7FEE770470000E5
:1034A00010B5104C0E48022120604FF4827060600D
:1034B0000020A060C4E90301012161614902C4E95F
:1034C000061020626062A0620720E0622046FFF7DB
:1034D000D5FA2068016841F04001016010BD00008C
:1034E00000300140D83E0020074908688268D24376
:1034F0009207FBD4FF22027308688168C943C90799
:10350000FBD1007B70470000D83E0020064A1168BE
:103510008B68DB439B07FBD4087310688168C94341
:10352000C907FBD1007B7047D83E0020074A1168CD
:103530008B68DB439B07FBD4087310688168C94321
:10354000C907FBD1007B024908707047D83E0020B4
:1035500009000020F0B515460E460746002405E098
:10356000385DFFF7D3FF3055641CA4B2AC42F7D3EB
:10357000F0BD7047FEF77EBF704710B5406A00216E
:10358000C185C184FFF7F8FB10BD70B5446A20689F
:10359000406994F84110C0F3C0100025212904D1DE
:1035A00018B1E584204600F0BFF82068406994F81F
:1035B0004210C0F38010222904D118B1E5852046BD
:1035C00000F08BF8606C40F0100060642046FFF75C
:1035D000D3FB70BD10B50146406A096809684FF019
:1035E000000289062ED4C28501680C3151E8003FE3
:1035F00023F4807341E80034002CF5D101681431C4
:1036000051E8003F23F0010341E80034002CF5D1DC
:103610000168143151E8003F23F0400341E80034D1
:10362000002CF5D1202180F84210016B012909D12D
:1036300001680C3151E8003F23F0100341E80034E9
:10364000002CF5D14263016B012902D0FFF74AFE3D
:1036500010BD818DFFF7CCFA10BD10B5406A012175
:103660004163016B012902D0FFF7B8FE10BD818DC7
:103670004908FFF7BDFA10BD10B5406A0021C185A9
:10368000202280F842200163FFF7B4FA10BD10B584
:103690000146406A09680968890616D40021C18478
:1036A0000168143151E8002F22F0800241E8002324
:1036B000002BF5D101680C3151E8002F42F0400297
:1036C00041E80023002BF5D110BDFFF7C5FE10BD6A
:1036D00010B5406AFFF7DEFE10BD01680C3151E8FD
:1036E000002F22F4907241E80023002BF5D10168ED
:1036F000143151E8002F22F0010241E80023002B91
:10370000F5D1016B012909D101680C3151E8002F75
:1037100022F0100241E80023002BF5D1202180F88F
:10372000421000210163704701680C3151E8002FFD
:1037300022F0C00241E80023002BF5D1202180F8BF
:103740004110704708B590F84210222901D002209C
:1037500008BD82684FF480539A4201D1016921B1BA
:10376000816A9A421BD04AB10AE00268816A5268B3
:10377000C2F308020A80816A891C08E0026972B1FA
:103780000268526802F07F020A70816A491C8162F5
:10379000C18D491E0904090CC18503D01BE00268D4
:1037A0005268F1E70168CA6822F02002CA60016825
:1037B000CA6822F48072CA6001684A6922F0010274
:1037C0004A61202180F8421000214163026B012AE6
:1037D00003D0FFF787FD002008BD016301680C31AD
:1037E00051E8002F22F0100241E80023002BF5D110
:1037F00001680A68D20602D50A6849680091818D7D
:10380000FFF7F6F9E7E7000070B5044600680169C4
:10381000E26821F44051114301612169A068084325
:10382000616908432168CA6841F20C639A43024304
:10383000CA6020684169A26921F440711143416165
:103840001E492068884202D1FEF752FF01E0FEF7D0
:103850003FFF00EBC00101EB0012606864218000B3
:10386000B2FBF0F3B3FBF1F36FF018067343B2FB56
:10387000F0F5B2FBF0F605EB8305322303EB0515FB
:10388000B5FBF1F5B6FBF1F605F0F00505EB061515
:10389000B2FBF0F6B2FBF0F0B0FBF1F06FF0180203
:1038A000504306EB800003EB0010B0FBF1F0216801
:1038B00000F00F002844886070BD0000003801400F
:1038C00038B5816204468285002013466064222256
:1038D00084F84220E56B1B4AAA62E56B1A4AEA6249
:1038E000E56B1A4A2A63E26B50630A462168E06B73
:1038F000091DFEF761FC206801684068009020699E
:1039000048B120680C3050E8001F41F4807140E855
:103910000012002AF5D12068143050E8001F41F051
:10392000010140E80012002AF5D12068143050E867
:10393000001F41F0400140E80012002AF5D10020AC
:1039400038BD0000D53500085B3600088B3500080F
:1039500038B50E480446FFF711FA0D49D1F8182181
:103960001068C043C0060FD4106850680090D1F8AA
:10397000602108685268C2F58072104408602046D1
:10398000BDE83840FFF7ACB938BD00001C07002087
:103990000406002038B50E480446FFF7EFF90D493C
:1039A000D1F818211068C043C0060FD410685068C1
:1039B0000090D1F8602108685268C2F50072104486
:1039C00008602046BDE83840FFF78AB938BD0000DE
:1039D000081A0020F0180020FEE7490050EAC12034
:1039E00018BF04204A0D18BF40F0010040F2FF72DA
:1039F000B2EB515F08BF40F00200012808BF05206C
:103A000070470907090E002804DB00F1E02080F868
:103A10000014704700F00F0000F1E02080F8141D42
:103A200070470000BFF34F8F05480168054A01F455
:103A3000E06111430160BFF34F8F00BFFDE700005D
:103A40000CED00E00400FA0530380A2801D201200C
:103A5000704700207047000070B51546084A1C46A4
:103A6000127882420BD807A001F009F921462846B6
:103A700001F00EF9BDE8704004A001F000B970BD7E
:103A8000080000205B25735D200000000D0A000087
:103A900010B50C4C01202070FEF7E6FC6168401A5E
:103AA000B0F57A7F0DD3227807484FF4807112B1B8
:103AB000FEF7CDFC02E00122FEF7D1FCFEF7D4FCBC
:103AC000606010BD000000200008014070B5B4B077
:103AD0006424214601A8FCF7D9FD34211AA8FCF77B
:103AE000D5FD342127A8FCF7D1FD7B480090A0F13B
:103AF0001403A0F1280279A101A8FCF7EFFB764896
:103B00007FA1283800F13C02B0F864301AA8FCF715
:103B1000E5FB714B7FA1283B03F1500227A8FCF77E
:103B2000DDFB81A000F03EFD0122824E55022946B8
:103B30003046FEF794FC4FF47A70FEF775FB0022D6
:103B400029463046FEF78BFC4FF47A60FEF76CFB9B
:103B50002046FEF769FB1E23082277A177A000F01C
:103B60006DFA08B176A0A1E001257AA000F01AFD57
:103B70002046FEF759FB7AA000F014FD1E23052213
:103B80006DA17AA000F05AFA08B17AA08EE07FA069
:103B900000F008FD2046FEF747FB80A000F002FD84
:103BA0001E23052281A183A000F048FA08B184A059
:103BB0007CE08AA000F0F6FC2046FEF735FB8BA0E7
:103BC00000F0F0FC1E2305225BA18DA000F036FA68
:103BD00008B18EA06AE094A000F0E4FC2046FEF755
:103BE00023FB95A000F0DEFC1E23052252A196A027
:103BF00000F024FA08B196A058E09BA000F0D2FC97
:103C00002046FEF711FB9CA000F0CCFC1E230522F1
:103C100049A19DA000F012FA08B19EA046E0A3A021
:103C200000F0C0FC2046FEF7FFFAA4A000F0BAFCAA
:103C30001E23052240A101A800F000FA08B1A3A0AC
:103C400034E0A9A000F0AEFC2046FEF7EDFAAAA0F1
:103C500000F0A8FC1E23052237A11AA800F0EEF9F7
:103C600008B1A9A022E0AFA000F09CFC2046FEF71E
:103C7000DBFAB0A000F096FC1E2305222EA1B2A014
:103C800000F0DCF908B1B5A010E0BBA000F08AFCA0
:103C90002046FEF7C9FABDA000F084FC1E230522D1
:103CA000BEA127A800F0CAF920B1BEA000F07AFC9E
:103CB000FFF7B8FE0A26C1A000F074FC2046FEF70C
:103CC000B3FA3146C1A000F06DFCC4480570C4A031
:103CD00000F068FC34B070BD583F002041542B4DBB
:103CE000434F4E4649473D222573222C22257322FD
:103CF0002C222573222C302C302C302C300000004C
:103D000041542B4D495053544152543D2225732266
:103D10002C25640041542B4D5355423D22257325DB
:103D200073222C3000000000D7BCB1B8B8B4CEBBB1
:103D300000000000001001404F4B00004154000003
:103D4000BFAABBFACAA7B0DCA3ACD7BCB1B8D6D85F
:103D5000C6F40000BFAABBFAB3C9B9A600000000B0
:103D6000B9D8B1D5BBD8CFD40000000041544530FC
:103D700000000000B9D8B1D5BBD8CFD4CAA7B0DCF9
:103D8000A3ACD7BCB1B8D6D8C6F40000B9D8B1D569
:103D9000BBD8CFD4B3C9B9A600000000D7BCB1B816
:103DA000B2E9D1AFBFA8D7B4CCAC00005245414472
:103DB0005900000041542B4350494E3F0000000081
:103DC000B2E9D1AFBFA8D7B4CCACCAA7B0DCA3AC22
:103DD000D7BCB1B8D6D8C6F400000000B2E9D1AF64
:103DE000BFA8D7B4CCACB3C9B9A60000D7BCB1B892
:103DF000C9E8D6C3B5A5C1ACBDD30D0A000000000B
:103E000041542B4349504D55583D3000C9E8D6C365
:103E1000B5A5C1ACBDD3CAA7B0DCA3ACD7BCB1B803
:103E2000D6D8C6F400000000C9E8D6C3B5A5C1AC19
:103E3000BDD3B3C9B9A60000D7BCB1B8C5E4D6C3D9
:103E4000CDF8C2E70000000041542B435354540006
:103E5000C5E4D6C3CDF8C2E7CAA7B0DCA3ACD7BCD3
:103E6000B1B8D6D8C6F40000C5E4D6C3CDF8C2E7D1
:103E7000B3C9B9A600000000D7BCB1B8BCA4BBEE62
:103E8000CDF8C2E70000000041542B43494943529A
:103E900000000000BCA4BBEECDF8C2E7CAA7B0DCAE
:103EA000A3ACD7BCB1B8D6D8C6F40000BCA4BBEE56
:103EB000CDF8C2E7B3C9B9A600000000D7BCB1B8BD
:103EC000C1ACBDD3B7FECEF1C6F70000C1ACBDD3C7
:103ED000B7FECEF1C6F7CAA7B0DCA3ACD7BCB1B869
:103EE000D6D8C6F400000000C1ACBDD3B7FECEF1F9
:103EF000C6F7B3C9B9A60000D7BCB1B8C1ACBDD331
:103F0000544350B6CBBFDA00C1ACBDD3544350B616
:103F1000CBBFDACAA7B0DCA3ACD7BCB1B8D6D8C681
:103F2000F4000000C1ACBDD3544350B6CBBFDAB3EC
:103F3000C9B9A600D7BCB1B8C5E4D6C3B1A3BBEE1E
:103F4000CAB1BCE40000000041542B4D434F4E4E1B
:103F50004543543D312C363000000000C5E4D6C343
:103F6000B1A3BBEECAB1BCE4CAA7B0DCA3ACD7BC5A
:103F7000B1B8D6D8C6F40000C5E4D6C3B1A3BBEE31
:103F8000CAB1BCE4B3C9B9A600000000D7BCB1B83F
:103F9000B6A9D4C4D6F7CCE2000000005355424184
:103FA000434B0000B6A9D4C4D6F7CCE2CAA7B0DC14
:103FB000A3ACD7BCB1B8D6D8C6F40000B6A9D4C457
:103FC000D6F7CCE2B3C9B9A600000000B5B1C7B0BE
:103FD000C0B4B5BDB2BDA3BA256400000000002086
:103FE000C1AACDF8B9FDB3CCD2BBC7D04F4B21008D
:103FF000F0B585B00F4800240294816941F01001AA
:1040000081618069012500F0100004904FF4007078
:10401000CDE90005084F0226694603963846FEF7AB
:1040200015F928028DE8710069463846FEF70EF949
:1040300005B0F0BD00100240001001402DE9F0472E
:104040001F4615468946804601261CE0414611A0C0
:1040500000F000FF3C460CE03220FEF7E5F800F0EF
:1040600063FF49460D48FCF779FA10B1002624B1E8
:1040700007E0641E14F0FF04EED1294608A000F00A
:1040800091FA6D1EEDB20DB1002EDFD13046BDE8C4
:10409000F087000025730D0A00000000EC170020D7
:1040A000B5DA2564B4CEB3ACCAB100002DE9F0474F
:1040B000002781463C463E46B8463DA1FCF74EFAF5
:1040C000801D054601463CA000F06CFA00206FF010
:1040D0002F0207E004EB840302EB43031944401C66
:1040E0008CB2C0B2295CA1F13003092BF2D9C8B25D
:1040F0002C2803D035A000F055FA0126374DB5F82D
:104100006E00A04205D136A000F04CFA0126B04660
:104110000AE0A5F86E40214634A000F043FA84225C
:104120002E49002000F0E2F834A14846FCF716FAC8
:10413000801D0446014633A000F034FAB8F1000FA8
:1041400008D034A000F02EFA224624493B4800F063
:1041500081FE2AE00021625CA2F13000092802D928
:10416000313819280ED8681890F87200904201D1A1
:104170007F1CFFB2491CC9B21029ECD3102F05D304
:10418000012612E02EA000F00DFAF9E76EB9002723
:10419000E919E05D81F8720084221049002000F0E6
:1041A000A5F87F1CFFB2102FF2D33046BDE8F08790
:1041B00022766572223A0000B0E6B1BEBAC5BAF303
:1041C000B5C4CAFDBEDDCEAA3A257300B0E6B1BEC5
:1041D000BAC5BDE2CEF6B4EDCEF30000303F00200C
:1041E000B0E6B1BEBAC5D6D8B8B40000D0C2B5C426
:1041F000B0E6B1BEBAC5CAC7256400002269642210
:104200003A2200006964BAF3B5C4CAFDBEDDCEAA85
:104210003A2573002A2A2A2A45525220B0E6B1BE16
:10422000BAC5D6D8B8B42CB7A2CBCDB3C9B9A6D627
:10423000B8C1EE204552522A2A2A2A00D453000837
:1042400069645B25645DB2BBCAC7D7D6B7FB2C696E
:10425000643D25640000000010B54FF0E0218A693C
:104260000C4B0D4C1B68B3FBF4F343439A4209D249
:1042700088699042FCD8981A4A698B69121A9A4246
:10428000FAD810BDD01A8B699342FAD28B69834257
:10429000F9D210BD1800002040420F0000F092B982
:1042A00010B507A000F07EF984210F48FCF7CCF987
:1042B0008422BDE810400C490020FFF7EFBF00004A
:1042C000B5B1C7B0CEAAD4CBD0D0C4A3CABD2CD769
:1042D000BCB1B8B4D3454550524F4DB6C1B3F64DFD
:1042E000515454D0C5CFA200303F00202DE9F041F9
:1042F000174606460D46002407E0295D304600F0CB
:1043000091F9761C641CF6B2A4B2BC42F5D3BDE8A8
:10431000F0810000F0B5154885B0816941F01001C9
:10432000816180694FF4006400F010000490112056
:10433000CDE900400E4F0325694603953846FDF749
:1043400085FF66000120CDE9006069460395384687
:10435000FDF77CFF012231463846FEF780F8012246
:1043600021463846FEF77BF805B0F0BD001002404C
:10437000001001402DE9F0472E4D814600244FF4F6
:104380008057224639462846FEF769F81420FFF781
:1043900063FF00264FF40068012239462846FEF7E5
:1043A0005EF81420FFF758FF6006040E41462846C9
:1043B000FEF748F808B1641CE4B21420FFF74CFF84
:1043C000002239462846FEF74AF81420FFF744FF3A
:1043D000761CF6B2082EDFD3B9F1000F1AD00022F6
:1043E000464641462846FEF73AF801223946284615
:1043F000FEF735F80220FFF72FFF00223946284646
:10440000FEF72DF8012231462846FEF728F820460F
:10441000BDE8F087012241462846FEF720F8012238
:1044200039462846FEF71BF80220FFF715FF002249
:104430003946E9E7001001402DE9F041144E0546E8
:104440004FF48057002239463046FEF708F8002422
:104450004FF40068EA0941463046FEF700F8680666
:10446000050E0220FFF7F8FE012239463046FDF71F
:10447000F6FF0220FFF7F0FE002239463046FDF736
:10448000EEFF641CE4B2082CE4D3BDE8F081000028
:104490000010014070B501220A4DD4022146284681
:1044A000FDF7DDFF012211032846FDF7D8FF0420A8
:1044B000FFF7D2FE21462846BDE870400022FDF7F6
:1044C000CEBF00000010014070B50B4D4FF40064EA
:1044D000002221462846FDF7C2FF0122110328468B
:1044E000FDF7BDFF0420FFF7B7FE21462846BDE8D3
:1044F00070400122FDF7B3BF001001402DE9F041EB
:104500000122154DD602002431462846FDF7A7FFAB
:104510000122170339462846FDF7A1FF0BE0641C72
:10452000E4B2FA2C04D9FFF7CFFF0120BDE8F081F7
:104530000220FFF791FE31462846FDF783FF002851
:10454000EDD1002239462846FDF789FF1420FFF7F8
:1045500083FE0020EAE700000010014030B585B07E
:10456000002002900D48816941F004018161806959
:104570004FF4807400F0040004900120CDE9004065
:104580000220074D039069462846FDF75FFE012291
:1045900021462846FDF763FF05B030BD00100240FC
:1045A000000801400FB405A110B503AB0220029A28
:1045B000FFF752FA10BC5DF814FB0000494E464F5D
:1045C000000000002DE9F04115460E460446FFF7B5
:1045D00061FFA020FFF730FFFFF790FF2046FFF7B5
:1045E0002BFFFFF78BFFFFF755FFA120FFF724FFFD
:1045F000FFF784FF00246F1E05E00120FFF7BAFEDD
:104600003055641CA4B2BC42F7DB0020FFF7B2FEB9
:10461000711901F8010CFFF757FFBDE8F0410520C3
:10462000FDF702BE70B50D460446FFF733FFA0202C
:10463000FFF702FFFFF762FF2046FFF7FDFEFFF7DF
:104640005DFF2846FFF7F8FEFFF758FFFFF73CFF36
:10465000BDE870400520FDF7E7BD0000FDF712FF43
:1046600000F0DEFA4FF4612000F01EFC4FF416500B
:1046700000F038FCFFF772FFFFF74CFEFFF7B8FCC5
:10468000FFF70EFE17A0FFF78DFF234C224923A052
:1046900034F8642F3C31FFF785FF1F4923A0FFF753
:1046A00081FF1D4925A01431FFF77CFF1A4927A07F
:1046B0002831FFF777FF618928A0FFF773FF1649BC
:1046C0002AA07231FFF76EFFFFF700FA00F0BCFC82
:1046D00000F0C8F900F028FC00F078FCFFF7D8F9EA
:1046E000F8E700002A2A2A2A2A2A2A2A2A2A2A2AF3
:1046F0002A2A2A2A2A2A2A2A4150502D436F6465E1
:104700002A2A2A2A2A2A2A2A2A2A2A2A2A2A2A2A09
:104710002A2A2A2A00000000303F0020B7FE20CEBF
:10472000F120C6F7A3BA25733A256400BFCDBBA715
:10473000B6CB4944A3BA257300000000D3C320BB05
:10474000A720C3FBA3BA257300000000C3DC202010
:104750002020C2EBA3BA257300000000CFB5CDB373
:10476000B0E6B1BEA3BA562564000000C9FDBCB6D0
:1047700020096964A3BA2573000000002DE9F04107
:1047800088B080460024142102A8FBF77FFF002692
:104790007B494046FBF7E2FE00287AD079A14046EB
:1047A000FBF7DCFE801D0546014678A0FFF7FAFE08
:1047B00002AF285DA0F13001092905D93139192945
:1047C00002D92031192903D8761C3855F6B207E0F2
:1047D000002672A0FFF7E6FE294679A0FFF7E2FE69
:1047E000641CE4B2122CE4D3122E02D377A0FFF79C
:1047F000D9FE7BA14046FBF7B1FE614C503C00283E
:104800002FD077A14046FBF7A9FEC07800250126EE
:10481000744F312806D0322824D0332845D034288C
:104820001FD161E070A14046FBF798FE48B170A02F
:10483000FFF7B8FE012202213846FDF710FE84F88A
:1048400067606EA14046FBF789FE00286AD06DA024
:10485000FFF7A8FE84F86750002202213846FDF7D2
:10486000FEFD5FE060A14046FBF778FE684F48B16F
:1048700068A0FFF797FE012204213846FDF7EFFDFF
:1048800084F868605DA14046FBF768FE002849D0C7
:1048900000E071E062A0FFF785FE002204213846A7
:1048A000FDF7DDFD84F868503CE04FA14046FBF782
:1048B00055FE48B15DA0FFF775FE0122082138467C
:1048C000FDF7CDFD84F869604CA14046FBF746FE3C
:1048D00040B359A0FFF766FE002208213846FDF7D5
:1048E000BEFD84F869501DE03FA14046FBF736FE4F
:1048F00048B154A0FFF756FE012210213846FDF7BB
:10490000AEFD84F86A603DA14046FBF727FE48B142
:104910004FA0FFF747FE002210213846FDF79FFD0C
:1049200084F86A501649842250390020FFF7DEFCD3
:1049300094F86A0000B1012094F8691001B10121D6
:10494000CDE9001094F8680008B1012300E00023CD
:1049500094F8670008B1012200E0002208493F48AE
:10496000503900F077FA3220FDF75EFC044902AAC4
:1049700050393B4800F06EFA08B0BDE8F081000005
:10498000803F0020226964223A0000004944C6F0BA
:10499000CABCCEBBD6C3CEAA257300004944D6D02C
:1049A000BBECD3D0B7C7B7A8D7D6B7FB2CBDABB23B
:1049B000BBBBE1B7A2CBCDB7B4C0A1CAFDBEDD0081
:1049C0004944D6B8D5EBCEAA257300004944D6D0C9
:1049D000D2BBC7D0D7D6B7FBD5FDB3A3000000002C
:1049E00022737700000C01407472756500000000AE
:1049F000BFAAB9D831B4F2BFAA00000066616C73D7
:104A000065000000BFAAB9D831B9D8B1D5000000FF
:104A100000140140BFAAB9D832B4F2BFAA00000006
:104A2000BFAAB9D832B9D8B1D5000000BFAAB9D849
:104A300033B4F2BFAA000000BFAAB9D833B9D8B1C5
:104A4000D5000000BFAAB9D834B4F2BFAA00000054
:104A5000BFAAB9D834B9D8B1D50000004C5300086A
:104A6000F05200082DE9F04186B052480026049625
:104A7000816941F008018161816901F008010091BB
:104A8000816941F0200181618069022400F02000E9
:104A900001270090CDE90247474D02A92846059419
:104AA000FDF7D4FB0420CDE90207DFF81081CDE942
:104AB000046402A94046FDF7C9FB0820CDE90207BE
:104AC000CDE9046402A92846FDF7C0FB1020CDE91A
:104AD0000207CDE9046402A92846FDF7B7FB384C6C
:104AE00094F8670008B1002200E001220221284664
:104AF000FDF7B5FC94F8680008B1002200E001223F
:104B000004214046FDF7ABFC94F8690008B100228F
:104B100000E0012208212846FDF7A1FC94F86A0074
:104B200008B1002200E0012210212846FDF797FC81
:104B300094F8670008B123A100E023A123A0FFF7A8
:104B400031FD94F8680008B11EA100E01EA124A068
:104B5000FFF728FD94F8690008B11AA100E01AA136
:104B600024A0FFF71FFD94F86A0008B115A100E02A
:104B700015A125A0FFF716FD94F86A0000B10120E9
:104B800094F8691001B10121CDE9001094F8680092
:104B900008B1012300E0002394F8670008B1012266
:104BA00000E0002206491D4800F054F906B0BDE8B7
:104BB000F081000000100240000C01400014014090
:104BC000303F0020BFAA0000B9D80000BCCCB5E738
:104BD000C6F731D7B4CCACCEAA3A2573000000009A
:104BE000BCCCB5E7C6F732D7B4CCACCEAA3A257365
:104BF00000000000BCCCB5E7C6F733D7B4CCACCED0
:104C0000AA3A257300000000BCCCB5E7C6F734D73C
:104C1000B4CCACCEAA3A2573000000004C53000877
:104C200030B58FB028216846FBF730FD14210AA863
:104C3000FBF72CFD01210804CDE9001000240294AB
:104C400002250491CDE907504FF4E0100990684621
:104C5000FDF784FD08B172B6FEE70F20CDE90A0525
:104C60004FF48060CDE90C4002210AA80E94FDF7B4
:104C700099FC002801D072B6FEE70FB030BD0FB42A
:104C800010B503A9029800F003F810BC5DF814FBFE
:104C900070B50A4601460F48FBF70EFB0E4DD5F8DE
:104CA00018010168C9434906FBD40024094E0BE0F2
:104CB000D5F81811305D4860D5F818010168C9436E
:104CC0004906FBD4641CA4B20248FBF759FCA0427D
:104CD000EED870BD040200201C00002010B5044670
:104CE00019A1FBF73BFC78B119A0FFF75BFCBFF300
:104CF0004F8F1E4801681E4A01F4E06111430160B4
:104D0000BFF34F8F00BFFDE71AA12046FBF726FC3B
:104D100028B11CA0FFF746FC2046FFF72FFD1DA180
:104D20002046FBF71BFC00280CD020A0FFF73AFC24
:104D30002046FFF7BBF9002804D0BDE810401FA0B3
:104D4000FFF730BC10BD0000434C4F5345440000FA
:104D5000D6F7BBFAB1BBC6C8CFC2CFDFA3ACD7BCB6
:104D6000B1B8D6D8C6F4A3A1000000000CED00E055
:104D70000400FA05696F742E70726F702E7365747B
:104D800000000000CAD5B5BDBFD8D6C6D6B8C1EEA2
:104D900000000000696F742E6F74612E7570677269
:104DA0006164652E706F737400000000CAD5B5BDD4
:104DB0004F5441C9FDBCB6D6B8C1EE00C9FDBCB662
:104DC0006964A3A8B0E6B1BEBAC5A3A9D6D8B8B4E1
:104DD000BBF26964B4EDCEF3A3ACBDABB2BBB8FC1F
:104DE000D0C2B3CCD0F20000F8B519480025A0F12C
:104DF000940400F16C01C4F80C01C4E94401E831E9
:104E0000016065602573FDF72FFBA06004F11000C1
:104E100000F16C01C4F88800C4E9230100F6D8163B
:104E200006604FF4006130462560FBF72FFC3146E9
:104E30004FF4807204F58C70FEF746FAD4F818012E
:104E4000016841680091C16841F01001C160F8BD7E
:104E5000980600200FB4124870B505AA0499FBF714
:104E60002BFA104DD5F818010168C9434906FBD447
:104E700000240B4E0BE0D5F81811305D4860D5F8D2
:104E800018010168C9434906FBD4641CA4B2044854
:104E9000FBF776FBA042EED870BC5DF814FB000077
:104EA000EC070020040600200C4910B50A4AE1E98D
:104EB0004620002088600822C860C1E90402886199
:104EC000C8610748FEF790F8002803D0BDE81040FD
:104ED000FCF752BF10BD0000003801401C0000204C
:104EE000340100200E4910B50C4AE1E946200020AB
:104EF00088600C22C860C1E904028861C861094861
:104F00000446FEF771F82046FEF76EF808B1FCF78C
:104F100033FFBDE81040FFF767BF000000440040CA
:104F2000040600201C07002010B51A4CD4E92210FA
:104F300088422DD003C8091A17A0FFF733FB40F2AF
:104F400001111F48FBF7A2FB54F88C0FD0E90012A7
:104F5000521A1B48FBF733FB19491AA0FFF722FB33
:104F6000206881880088081A81B21548FFF7B6FECC
:104F70004FF480711448FDF76AFA20680C3001C4C0
:104F800054F89019884203D102481030C4F88C00BC
:104F900010BD000004060020B4AEBFDA32B1BEB4CA
:104FA000CEBDD3CAD52564D7D6BDDAB1A8CEC4CA82
:104FB000FDBEDD282A3447C4A3D7E92A29A3BA00B5
:104FC000EC170020257300000008014010B5144CB8
:104FD000D4E94310884222D0217B00291FD103C885
:104FE000091A10A0FFF7DEFAD4F8100182880168D0
:104FF000501A82B204F58C70FEF7F2F900280ED137
:1050000001202073D4F810010C30C4F81001D4F83A
:105010001411884203D104F19400C4F8100110BDAA
:1050200004060020B4AEBFDA32B1BEB4CEB7A2CB14
:10503000CD2564D7D6BDDACAFDBEDD282A3447C4E3
:10504000A3D7E92A29000000154810B5816986B068
:1050500041F0040181618069124C00F00400049069
:1050600010200090012001900290032003906946D7
:105070002046FDF7EBF8012210212046FDF7EFF95D
:10508000FEF70EFA00F01AF8A0F56F41163903D0BA
:1050900005A0FFF787FAFEE700F050F806B010BD54
:1050A0000010024000080140B6C1C8A15732355176
:1050B0003634CAA7B0DCA3A1000000001FB510A1C0
:1050C000D1E90001CDE9000100F020F80E4C0022EA
:1050D00010212046FDF7C3F9062202A96846FEF713
:1050E00039FA012210212046FDF7B9F99DF80D008B
:1050F0009DF80C1004B000EB012080B210BD000040
:1051000090000000000000000008014070B50A4C4B
:10511000002210212046FDF7A2F90520FEF706FA2D
:10512000FEF7E2F90546012210212046FDF797F926
:10513000E807EDD170BD00000008014010B5FFF791
:10514000E5FF084C002210212046FDF788F90620D3
:10515000FEF7ECF920460122BDE810401021FDF7D2
:105160007EB900000008014010B500290AD0087877
:10517000002807D005487844FCF7CCF9002801D076
:10518000002010BD0248784410BD0000020300005A
:10519000FA02000010B500290AD00878002807D0CC
:1051A00005487844FCF7B6F9002801D0002010BD6E
:1051B0000248784410BD0000F2020000EA0200003C
:1051C000FBF7D4BDFBF708BF010202030405060785
:1051D00008090A0B0C0D0E0F101000000000000053
:1051E0000000010203040607080900000000010294
:1051F0000304040000080000000000000002000199
:1052000000001000000000000000000030313233C8
:1052100034353637383941424344454640305800EA
:10522000303132333435363738396162636465661C
:1052300040307800303132333435363738396162B6
:105240006364656678700030313233343536373810
:105250003941424344454658500000000240000096
:10526000000000A00000000005400000000000C891
:10527000000000000C4000000000409C0000000006
:10528000194000000020BCBE0000000034400000B7
:10529000BFC91B8E00000004B5400000504BCFD0AA
:1052A0006607E2CF010000006C4100003E8251AA77
:1052B000DFEEA73401000000D9420000DCB5A0E217
:1052C0003A301F97FFFFFFFFB4450000FD25A0C83F
:1052D000E9A3C14FFFFFFFFFFF3F00000000008078
:1052E00000000000FF3F0000000000800000000000
:1052F00041542B4D5055423D222F696F742F6461EC
:1053000074612F75702F2573222C302C302C227B4A
:105310005C323269645C32323A5C323225735C3220
:10532000322C5C3232636F64655C32323A302C5C12
:1053300032326D6573736167655C32323A5C32326A
:105340004F4B5C32327D220D0A00000041542B4D40
:105350005055423D222F696F742F646174612F751F
:10536000702F2573222C302C302C227B5C3232683B
:1053700065616465725C32323A5C3232696F742EF8
:1053800070726F702E706F73745C32322C5C3232BC
:10539000626F64795C32323A7B5C32327377315CB3
:1053A00032323A25642C5C32327377325C32323AD4
:1053B00025642C5C32327377335C32323A25642CAC
:1053C0005C32327377345C32323A25647D7D220D53
:1053D0000A00000041542B4D5055423D222F696F69
:1053E000742F646174612F75702F2573222C302CFB
:1053F000302C227B5C32326865616465725C3232CB
:105400003A5C3232696F742E6F74612E70726F67FE
:10541000726573732E706F73745C32322C5C32322F
:10542000626F64795C32323A7B5C323269645C323E
:10543000323A5C3232252E3136735C32322C5C3299
:105440003270726F67726573735C32323A31307DDD
:105450007D220D0A00000000A45500080000002075
:105460001C0000006C010008C05500081C00002052
:10547000FC450000880100081C00000043000000FB
:10548000F8FFFFFF0C0000000E0000000F000000FE
:105490002E0000001001000043000000F8FFFFFF95
:1054A0000040404040404040404041414141414037
:1054B00040404040404040404040404040404040EC
:1054C000400502020202020202020202020202027B
:1054D0000220202020202020202020020202020280
:1054E00002029090909090901010101010101010D8
:1054F00010101010101010101010101002020202E4
:105500000202888888888888080808080808080827
:105510000808080808080808080808080202020223
:10552000400000000000000000000000000000003B
:10553000000000000000000000000000000000006B
:10554000000000000000000000000000000000005B
:10555000000000000000000000000000000000004B
:10556000000000000000000000000000000000003B
:10557000000000000000000000000000000000002B
:10558000000000000000000000000000000000001B
:10559000000000000000000000000000000000000B
:1055A00000000000000000000000000001000000FA
:1055B0000100000010000000000000000024F400C2
:0400000508000131BD
:00000001FF
